:1000000012C018951895189518951895D1C118957E
:100010001895189518951895189518951895189578
:100020001895189518958FED8DBFC0ECE4EB4E2E0A
:10003000DD275D2EEEE7F0E0A0E6B0E088278D93A7
:100040003197E9F784B7082E877F84BF8FE181BDA0
:1000500087E081BD662483EE87BB8FEF81BB8DEF88
:1000600088BB8FEF82BB81E083BF80E080BF86E0EA
:1000700082BF89B7826089BFEEE3F6E0E6D281E015
:1000800090E0AFE68D939C93AFE60D911C910A3002
:1000900050E0150710F009F00CC0DAD2AFE6AD90D1
:1000A000A0E7AA0D49D30C92D0D2AFE6D4D208F47F
:1000B000EBCF80E08093600080E080936100ACE74C
:1000C0003FD3809165008F7D80936500EAE0F0E08A
:1000D000ACE691E056D3E4E1F0E0ADE691E051D337
:1000E000EEE1F0E0ABE891E04CD300918B000E3CE8
:1000F00008F004C085B7816285BF8895809165004E
:1001000080688093650080E080938A0081E083BFEF
:100110007894BC98A5E69C9194FF04C0B49B0EC053
:100120009F7E9C93B4990AC08AE09F939927F5D249
:100130009F91B49903C090619C9320D2BA98A5E690
:100140009C9193FF04C0B29B0EC0977F9C93B29981
:100150000AC08AE09F939927E0D29F91B29903C089
:1001600098609C931ED2BB98A5E69C9192FF04C018
:10017000B39B0EC09B7F9C93B3990AC08AE09F9368
:100180009927CBD29F91B39903C094609C931ED2C0
:1001900000916D000E3109F003C08DE180936D0078
:1001A00000916D000F3F09F003C080E080936D0067
:1001B00000916C00063009F003C085E080936C006C
:1001C00000916C000F3F09F003C080E080936C0049
:1001D00000918A00003009F006C000916C004AE0EE
:1001E000D7D2A3E64C9300918A00013009F004C0F5
:1001F00080916D0080936400A5E68C9186FB0EF0E3
:10020000D4C0809165008F7B80936500009162006F
:10021000003009F033C0A2E80D911C9141E050E09C
:10022000040F151FAFE60D931C93AFE6AD90A0E74A
:10023000AA0D8C9182BBC59AA5E68C9185FB0EF028
:100240001DC0ACE70D911C9148EE53E030D2A8E8F8
:100250004D935C93A8E80D911C9148EE53E041D278
:10026000AFE60D931C93ACE70D911C91AFE64D9159
:100270005C91041B150BA8E60D931C930091620082
:10028000013009F03AC0A4E80D911C9141E050E022
:10029000040F151FAFE60D931C93AFE6AD90A0E7DA
:1002A000AA0D8C9182BBC09AC79800918A00003039
:1002B00009F001C0C098A5E68C9185FB0EF01DC029
:1002C000A8E60D911C9144E650E0F1D1A6E84D93CB
:1002D0005C93A6E80D911C9144E650E002D2AFE693
:1002E0000D931C93A8E60D911C91AFE64D915C9186
:1002F000041B150BAAE60D931C93009162000230BB
:1003000009F03BC0A6E80D911C9141E050E0040FBC
:10031000151FAFE60D931C93AFE6AD90A0E7AA0DB5
:100320008C9182BBC09AC79AC69800918A0001300E
:1003300009F001C0C098A5E68C9185FB0EF01DC0A8
:10034000AAE60D911C914AE050E0B1D1A4E84D938A
:100350005C93A4E80D911C914AE050E0C2D1AFE655
:100360000D931C93AAE60D911C91AFE64D915C9103
:10037000041B150BA2E80D931C930091620003303F
:1003800009F013C0A8E80D911C9141E050E0040F62
:10039000151FAFE60D931C93AFE6AD90A0E7AA0D35
:1003A0008C9182BBC09AC69AC598B3CEF894FFCF01
:1003B0000F921F922F923F924F925F927F92AF9235
:1003C000BF920F931F932F933F934F935F936F931E
:1003D0007F938F939F93AF93BF93CF93DF93EF93CD
:1003E000FF938FB78F93F894A0E68C918F5F8C93D7
:1003F000009160000A3010F009F001C0A2C080E056
:100400008093600080916500806480936500A2E61F
:100410008C918F5F8C9300916200033010F009F093
:1004200001C01EC080E080936200A6E614D1A6E65B
:100430000D911C91033651E0150709F00CC0A6E69A
:100440007FD1A5E68C9187FB0EF405C080916300F7
:10045000815080936300809165008F7D809365005B
:10046000A1E68C918F5F8C9300916100083C10F0A5
:1004700009F001C066C080E08093610000918A00AD
:10048000023009F03FC0009163000F3F09F008C03F
:10049000809164008150809364008BE380936300BB
:1004A000B49905C0809165008F7780936500A5E6BB
:1004B0008C9187FB0EF401C0C19AB29905C080915E
:1004C0006500806880936500A5E68C9187FB0EF03F
:1004D00001C0C19800916400003081E009F080E023
:1004E0008F9300916300003081E009F080E09F91DC
:1004F0008923882309F406C0C1988091650080682B
:1005000080936500A4E60D91112744E650E0E9D000
:10051000AEE70D931C93A3E68C91A0E88D938827FA
:100520008C93AEE70D911C91A0E84D915C91040F66
:10053000151FACE70D931C9380916500806280933A
:10054000650078948F918FBFFF91EF91DF91CF91EC
:10055000BF91AF919F918F917F916F915F914F91DB
:100560003F912F911F910F91BF90AF907F905F901F
:100570004F903F902F901F900F90189500918A00F8
:10058000003009F004C0ACE68C918F5F8C93009131
:100590008A00013009F004C0ADE68C918F5F8C9326
:1005A000089500918A00003009F005C080916C0028
:1005B000815080936C0000918A00013009F005C0E1
:1005C00080916D00815080936D000895F894AAE8A1
:1005D0008C918F5F8C9300918A00023009F025C0C6
:1005E00000916C004AE0D4D0A3E64C9380916D005A
:1005F0008093640080916D0080936E00EAE0F0E0EB
:10060000ACE691E07BE7ACD0E4E1F0E0AEE691E06F
:100610007BE7A6D080918B00815080938B00EEE128
:10062000F0E0ABE891E07BE79BD000918A000330DB
:1006300009F003C080E080938A0078940895015DFA
:1006400012184C28601D000C7E008E2E9F2E0895DF
:10065000E82DF92D0895ED91FC91EF5FFF4FFC938C
:10066000EE93089508D03DD000FC10D0089503D03B
:100670001ED001F8F9CF0024E89457FF02C009D03A
:10068000689400F80BD010F80124089502D009D026
:100690000895509540954F5F5F4F0895E89417FF78
:1006A0000895009510950F5F1F4F68940895352F9A
:1006B000242FE894452B11F468940895512F402F6E
:1006C0000027112780E1440F551F001F111F021B37
:1006D000130B416018F4020F131F4E7F8A9599F790
:1006E0000895752F642F55274427FF93F1E18894CF
:1006F00005C010F4460F571F569547951795079557
:10070000FA95B9F7FF9108953197F1F70895689434
:1007100062F80895E89462F80895EF93FF93EE2746
:10072000E82BE92B31F0E8EEF3E03197F1F7019790
:10073000D1F7FF91EF910895C89531960020089563
:1007400082E001C084E099279D938A95E9F7089596
:10075000E199FECFEEBB3196089591E001C092E0A1
:100760007B3751F47FB7F894F3DF8D918DBBE29A1C
:10077000E19A9A95C9F77FBF7727089591E001C064
:1007800092E0E6DFE09A8DB38D939A95D1F70895C4
:10079000FF935527F8E0469508F4500F5795479575
:0807A000FA95D1F7FF910895CD
:00000001FF
